:1008ED0000C000F900A400B000990092008200F849
:1008FD00008000900088008300C600A10086008E55
:030AEC005401FFB3
:0A0AEF00E51125E0F511EF42112298
:0D0AF900E51125E0F511EFF4540142112242
:040BE400EF52112299
:070BA100EFF4540152112290
:040BE800EF421122A5
:070BA800EFF4540142112299
:0E0AB400E511F45401FFE51154FE4FF5112237
:060BD200E5115401FF22B1
:0D0B0600E511C313FFE51154015FF5112245
:0D0B1300E511C313FFE51154014FF5112248
:0E0AC200E51125E0F511EDF45F54014211221B
:0E0AD000E51125E0F511EFF45D54014211220D
:08000300EDF45F5401521122DB
:080B8900EFF45D54015211224A
:080B9100EDF45F540142112252
:080B9900EFF45D54014211224A
:070BAF00EDF45F5401FF2289
:070BB600EFF45D5401FF2282
:0D0B2000E51825E0FFE51154014FF51822FE
:0D0B2D00E5185401FFE51154FE4FF51122AB
:1009A500E5185401FFE51154FE4FF511E518C31381
:0309B500F5182210
:100A95008E5E8F5FE55F2DFFE55E3C8FF00204966D
:1009B8008E608F61C3E5619DFFE5609C8FF0020446
:0109C8009698
:090B80001203D5EE8FF002049679
:0F0AA5008B5B8A5C895D1203E7EE8FF00204968B
:070BBD00E475F00102045E83
:070BC40074FFF5F002045E6E
:1009C9008E628F63E5625CFFE5635DCF8FF00204A1
:0109D9009687
:1009DA008E648F65E5644CFFE5654DCF8FF00204A8
:0109EA009676
:1009EB008E668F67E5666CFFE5676DCF8FF002044F
:0109FB009665
:1009FC00EFF4FFEEF4FEEF2401FFE43E8FF002046F
:010A0C009653
:060BD800EFF45401FF22BE
:060BDE00EE8FF002049608
:0A0B7600EFF4FFEEF48FF002049696
:100897008B4B8A4C894D120433FFAEF0AB4EAA4FF7
:1008A700A950120433FDAB4BAA4CA94DE5F08DF0CE
:0F08B700120496AB4EAA4FA950EE8FF002049692
:10050A008E528F538B548A5589567C037DE8120389
:10051A00E7EFC454F07B00FAAE52AF537C037DE898
:10052A001203E78C528D53AE52AF537C007D641296
:10053A0003E7EFFEE4EE4202AE52AF537C007D6465
:10054A001203E78C528D53AE52AF537C007D0A12D0
:10055A0003E7EFC4F8540FC868FFEEC454F048FE2E
:10056A00EFFBEE4202AE52AF537C007D0A1203E764
:10057A008C528D53E5524AFFE5534BAB54AA55A909
:07058A0056CF8FF00204962A
:10068C008E578F58E558780CCEA2E713CE13D8F8B6
:10069C007E00540FFF7C037DE81203D58E598F5AD0
:1006AC00E557FF3395E07E00EF540FFF7C007D642F
:1006BC001203D5EF255AF55AEE3559F559E558AED2
:1006CC00577804CEA2E713CE13D8F87E00540FFF50
:1006DC007C007D0A1203D5EF255AF55AEE3559F5F3
:1006EC0059E558540F255AF55AE43559F559855A98
:0406FC00F00204966E
:10090D00E51125E0F511C3EF9DEC6480F8EE6480F0
:0B091D00984004431101225311FE22F8
:10092800E51125E0F511D3EF9DEC6480F8EE6480C5
:0B093800985004431101225311FE22CD
:10094300E51125E0F511D3EF9DEC6480F8EE6480AA
:0B095300984004431101225311FE22C2
:10095E00E51125E0F511C3EF9DEC6480F8EE64809F
:0B096E00985004431101225311FE2297
:10097900E51125E0F511EF6D7002EE6C600443118D
:0609890001225311FE22C1
:10098F00E51125E0F511EFB50508EEB504044311A7
:06099F0001225311FE22AB
:100A0D00C3EF9DEC6480F8EE64809850035311FEA3
:010A1D0022B6
:100A1E00D3EF9DEC6480F8EE64809840035311FE92
:010A2E0022A5
:100A2F00D3EF9DEC6480F8EE64809850035311FE71
:010A3F002294
:100A4000C3EF9DEC6480F8EE64809840035311FE80
:010A50002283
:0C0B3A00EFB50507EEB504035311FE22D1
:0C0B4600EF6D7002EE6C60035311FE2294
:100A5100C3EF9DEC6480F8EE64809840034311017C
:010A61002272
:100A6200D3EF9DEC6480F8EE64809850034311014B
:010A72002261
:100A7300D3EF9DEC6480F8EE64809840034311014A
:010A83002250
:100A8400C3EF9DEC6480F8EE648098500343110139
:010A9400223F
:0C0B5200EF6D7002EE6C60034311012295
:0C0B5E00EFB50507EEB5040343110122BA
:070BCB00E4FF0FBF0AFC224A
:10086700E4FEC2B4120BCBC2B3120BCBD2B3120B42
:10087700CBD2B4120BCBE4FDEE25E0FE309403435C
:100887000601C2B3120BCBD2B30DBD08EBAF0622E4
:1001F4000510E510C394054003E4F510E510146000
:100204005B1470030202B01470030202FC24036046
:100214000302034E7C0090000DE0540FFD25E0FF27
:10022400EC33FE74ED2FF58274083EF583E493FC01
:10023400740193FD43040890010AE0FFC4131313EF
:10024400540130E0057DFF0203A4EF131313541F80
:1002540020E0030203A453057F0203A490000CE0F2
:10026400FEA3E07804CEA2E713CE13D8F87C0054A2
:100274000FFD25E0FFEC33FE74ED2FF58274083E8C
:10028400F583E493FC740193FD43040490010BE0B3
:1002940030E0057DFF0203A490010AE0FFC4540F7F
:1002A40020E0030203A453057F0203A490000CE0A2
:1002B400FF3395E07C00EF540FFD25E0FFEC33FEA7
:1002C40074ED2FF58274083EF583E493FC74019376
:1002D400FD43040290010BE0FFC31330E0057DFFF2
:1002E4000203A490010AE0FFC413540720E00302B0
:1002F40003A453057F0203A490000CE0FEA3E0785E
:100304000CCEA2E713CE13D8F87C00540FFD25E0E1
:10031400FFEC33FE74ED2FF58274083EF583E4930D
:10032400FC740193FD43040190010BE0FF1313548B
:100334003F30E0047DFF806890010AE0FFC413139E
:10034400540330E05B53057F805690010BE0F9C401
:100354001313540175F008A4FBAAF0E9C413131392
:10036400540175F010A4FFE5F04AFAEF4BFBE9C421
:1003740013540175F004A4FFEA45F0FAEB4FFBE9CE
:10038400C4540125E0FFE4334AFEEB4FFFE91313A5
:10039400135401FBEEEF4BF4FFEEF47410FCAD07C5
:1003A4007B10C2B3120BCBEC20E704C2B78002D29D
:1003B400B7120BCBED25E0FDEC33FCD2B3120BCB23
:1003C400DBE0D2B7120BCBC2B5120BCBD2B5020B0A
:0103D400CB5D
:10000E00E52E70030201F3152E0517E517B405173B
:10001E00AF30EFC4135401F45401FFC43354E0FF66
:10002E00E53054DF4FF530E517B40A1CAF30EFC49E
:10003E00135401F45401FFC43354E0FFE53054DF90
:10004E004FF530051DE4F517E4F552E55213131381
:10005E00541F2412F8E6FD7C00E5525407FF74018C
:10006E007E00A807088005C333CE33CED8F9FFEE45
:10007E005CFEEF5D4E6043E55225E025E0246EF513
:10008E0082E43400F583E0FEA3E0FFE55225E0258F
:10009E00E0246CF582E43400F583E0FCA3E0C39F1A
:1000AE00EC9E5016E55225E025E0246CF582E434F2
:1000BE0000F583E475F00112041DE55225E025E0FC
:1000CE00246EF582E43400F583E0FEA3E0FFE552F2
:1000DE0025E025E0246CF582E43400F583E0FCA3F2
:1000EE00E0C39FEC9E407AE55225E025E0246CF5B6
:1000FE0082E43400FEC3E582946CFFEE9400FE7C35
:10010E00007D021203E77C007D021203E77C007D76
:10011E00081203E7741E2FF8C000E6FFC007E55271
:10012E0025E025E0246CF582E43400FEC3E58294DC
:10013E006CFFEE9400FE7C007D021203E77C007DD6
:10014E00021203E77C007D081203E7AF057401A8D5
:10015E0007088002C333D8FCFED0E04ED000F680F4
:10016E0079E55225E025E0246CF582E43400FEC3E7
:10017E00E582946CFFEE9400FE7C007D021203E794
:10018E007C007D021203E77C007D081203E7741EDB
:10019E002FF8C000E6FFC007E55225E025E0246CED
:1001AE00F582E43400FEC3E582946CFFEE9400FE0B
:1001BE007C007D021203E77C007D021203E77C00C7
:1001CE007D081203E7AF057401A807088002C33348
:1001DE00D8FCF4FED0E05ED000F60552E552642065
:0601EE006003020059222B
:1007AD00E51DB41E19AF30EFC413135401F45401F9
:1007BD00FFC4333354C0FFE53054BF4FF530E51D52
:1007CD00B43C1CAF30EFC413135401F45401FFC4F7
:1007DD00333354C0FFE53054BF4FF530E4F51D22DF
:03000B00020700E9
:10070000C0E0C0D075D008758CEEAF30EF13131376
:100710005401F45401FF33333354F8FFE53054F7F8
:100720004FF530053AE53A30E0020516E53AB40AED
:1007300015AF30EFC45401F45401FFC454F0FFE589
:100740003054EF4FF530E53AB4141AAF30EFC454DB
:1007500001F45401FFC454F0FFE53054EF4FF5307D
:0A076000052E753A00D0D0D0E0322B
:10076A007594FF752F05E4F530F53190000CF0A370
:10077A00F090010BE054F7F054EFF054DFF054BF5F
:10078A00F0547FF090010AE054F7F054EFF054DF90
:10079A00F054BFF0547FF0A3E054FEF054FDF0543F
:0307AA00FBF0223F
:040BEC00752F092236
:1007ED00E4FFEF25E025E0246CF582E43400F58389
:1007FD00E4F0A3F00FBF20EAE4FF7F4090002CE46B
:10080D00F0A3DFFCE4FF741E2FF8E4F60FBF04F62F
:0D081D00E4FF74192FF8E4F60FBF04F62273
:0E0ADE00758911D2B4D2B9D2A9D28CD2AF226E
:10082A00AFA0EFC3135455FEEF25E054AA4EFF13B1
:10083A00135433FEEF25E025E054CC4EFF54F0FE6E
:10084A00E590540F4EF4F522EF540FF4540FF523AC
:0D085A00120867EFF4F5248528800201F4F0
:10059100E4FF74222FF8E6FE743F2FF8A6060FBF82
:1005A10006F0E4FF74282FF8E6FE74452FF8A6063E
:1005B1000FBF06F0E4FF74682FF8E6FE74202FF5F4
:1005C10082E43401F583EEF00FBF20EAE4FF74EC1E
:1005D1002FF582E43400F583E0FE74402FF582E4C8
:1005E1003401F583EEF00FBF20E4E4FF741E2FF811
:1005F100E6FE74362FF8A6060FBF04F0E4FF741967
:0F0601002FF8E6FE74322FF8A6060FBF04F02282
:1008C60075510112076A1207ED120ADE12082A1282
:1008D600061012000E1207AD120591E55160EDE407
:0708E600F551120BEC80E557
:10061000E522120AECE51130E01EAF12EFC3132001
:10062000E023EF4402F512E4900070F0A3F0A3740D
:1006300002F0A37458F0800DE51254FDF512E49019
:100640000070F0A3F0120BD2EF5401FFE52854FE26
:100650004FF528AF1EEFC313120AEC120BD2EF5462
:1006600001FF25E0FFE52854FD4FF528E52F540153
:10067000FF120AEFE51130E011900070E0FEA3E0F8
:0C068000FF7B017A00790C12050A0022B1
:03000000020B6A86
:0C0B6A00787FE4F6D8FD7581870208C68C
:1003D500EF8DF0A4A8F0CF8CF0A428CE8DF0A42E3C
:0203E500FE22F6
:1003E700C2D5EC30E709B2D5E4C39DFDE49CFCEE31
:1003F70030E715B2D5E4C39FFFE49EFE1204B5C3F0
:10040700E49DFDE49CFC80031204B530D507C3E4EA
:060417009FFFE49EFE229F
:10041D00C5F0F8A3E028F0C5F0F8E582158270026A
:06042D001583E038F02207
:10043300BB010A89828A83E0F5F0A3E02250068794
:10044300F009E71922BBFE07E3F5F009E319228956
:0B045300828A83E493F5F07401932289
:10045E00BB010789828A8302041D500B09C5F02750
:10046E00F7C5F01937F722BBFE0D09F8E325F0F3B7
:10047E00C5F019E338F322F889828A837401932533
:08048E00F0C5F0F8E4933822F8
:10049600BB010A89828A83F0E5F0A3F0225006F7B1
:0F04A60009A7F01922BBFE06F3E5F009F31922AE
:1004B500BC000BBE0029EF8DF084FFADF022E4CC2B
:1004C500F875F008EF2FFFEE33FEEC33FCEE9DECF4
:1004D500984005FCEE9DFE0FD5F0E9E4CEFD22ED3A
:1004E500F8F5F0EE8420D21CFEADF075F008EF2F84
:1004F500FFED33FD4007985006D5F0F222C398FD75
:050505000FD5F0EA2211
:00000001FF
